:0200000480007A
:100000006F004005732F2034930F8000630AFF03B5
:10001000930F90006306FF03930FB0006302FF038A
:10002000170F0000130F4F2C63040F0067000F0021
:10003000732F203463540F006F00400093E19153FD
:10004000171F000023203FFC171F0000232E0FFA6C
:100050006FF01FFF930000001301000093010000E8
:10006000130200009302000013030000930300003A
:100070001304000093040000130500009305000022
:10008000130600009306000013070000930700000A
:1000900013080000930800001309000093090000F2
:1000A000130A0000930A0000130B0000930B0000DA
:1000B000130C0000930C0000130D0000930D0000C2
:1000C000130E0000930E0000130F0000930F0000AA
:1000D000732540F16310050097020000938202012E
:1000E000739052307350447497020000938202015F
:1000F00073905230735000189702000093824202AE
:10010000739052309B021000939252039382F2FF3D
:100110007390023B9302F0017390023A73504030A7
:100120009702000093824201739052307350203046
:100130007350303093010000970200009382C2ECAC
:1001400073905230130510001315F501635C050020
:100150000F00F00F930110009308D0051305000065
:100160007300000093020000638A02007390521033
:10017000B7B200009B82921073902230735000300F
:10018000372500001B05058073200530970200000D
:100190009382420173901234732540F17300203032
:1001A0009301200017050000130545017315553014
:1001B0009305800073A0557A731055307310007A40
:1001C000F325007A6316B0101706000013064602E6
:1001D0007310267A1B0510001315D503130545046B
:1001E0007310157AF325107A6318B5006304000CB8
:1001F0009301300003250600930140001B05100009
:100200001315D503130515047310157AF325107A09
:100210006310B502172600001306C6DE7310267A97
:1002200003260600630806089301500023200600F9
:10023000930160001B0510001315D5031305250459
:100240007310157AF325107A6314B5062320C600BF
:100250009301700003260600631E060413051000B8
:100260007310057AF325007A6314B5061B05100098
:100270001315D503130515047310157A972600007E
:10028000938686D87390267A9301800083A6060011
:10029000638206029301A00017260000130686D68B
:1002A0002320C6009301B000032606006314060055
:1002B000631030020F00F00F638001009391110072
:1002C00093E111009308D00513850100730000002D
:1002D0000F00F00F930110009308D00513050000E4
:1002E0007300000093F21100E39602FC93023000C9
:1002F00073232034E39062FCF32210349382420093
:100300007390123473002030731000C0000000009E
:1003100000000000000000000000000000000000DD
:1003200000000000000000000000000000000000CD
:1003300000000000000000000000000000000000BD
:1010000000000000000000000000000000000000E0
:1010100000000000000000000000000000000000D0
:1010200000000000000000000000000000000000C0
:1010300000000000000000000000000000000000B0
:081040000000000000000000A8
:1020000000000000000000000000000000000000D0
:040000058000000077
:00000001FF
